:1000000008308A0000280000FF00030E8301A100D1
:100010007F08A0000A08A8008A01A00E0408A20018
:100020007708A3007808A4007908A5007A08A6003C
:100030007B08A700831383128C308400801C222845
:100040008C183528220884002308F7002408F800BB
:100050002508F9002608FA002708FB0028088A006E
:10006000210E8300FF0E7F0E09008A1149280A1015
:100070008A100A1182074C343A342034253455341E
:100080002034203452343A3420342534553400346A
:100090000034420F4C284E280130C20743080E3C62
:1000A0000318C30A4608553C0318C60AC708031DAF
:1000B000C7038C108A11222812308316A402031C55
:1000C0006F28A4308400FC3080050310800C800C65
:1000D000000803196F286D280000800B6C2883121C
:1000E000003483162108A3002008A200A208031DE3
:1000F0007C28A30803199B28051383120517831670
:100100008513831285137C088316A40083125C2058
:10011000831685138312851783160513831205131F
:100120007C088316A40083125C208316220803191E
:10013000A303A2037628831200347D3084000008D4
:100140000319B1280130F800F701F70BA528F80BC7
:10015000A4284A30F700F70BAB2800000000800B02
:10016000A228003470088400831620088000840AC6
:100170008001F00A8312003483162108F80120025E
:100180000318C5282008F700D128F7010830A2007D
:10019000A00DF70D210877020318F700F80DA20B48
:1001A000C828831200347E13FE127D088316A00037
:1001B0006430A1008312BC207708FD007808031D7D
:1001C0000129FE1A0129FE1913297E1BED287E182C
:1001D000ED287E19ED28FE1B13297E1CF928FE1B35
:1001E00013297E1BF9287E1813297E19F928FE1B76
:1001F000132920307E1E30308316A0008312B220D7
:100200001329FE16FE1F0D2978088000F8002D30F6
:100210008316A0008312B220FE13303078078316B5
:10022000A0008312B2207E1B20297D088316A00027
:100230000A30A1008312BC207708FD007E17DE285B
:10024000FE1F27292D308316A0008312B2203030E4
:100250007D078316A0008312B2200034BC01391C34
:1002600033293910342939140034391C6029831694
:100270008511831285154930F700F70B3D290000E1
:10028000000083168511831285114930F700F70BA2
:100290004729000000008316851183128515493017
:1002A000F700F70B51290000000083168511831217
:1002B00085111930F700F70B5B2900000000722947
:1002C00083168511831285158930F700F70B66298F
:1002D00083168511831285117230F700F70B6E2992
:1002E0000000000000348316A0012008073C031C16
:1002F000CF297E080139A1008312BE080319822983
:100300000030832901308316A2008312BD0803192F
:100310008B2900308C29013083162205003A0319FD
:10032000A4292108A20003108312BB0CBA0C0308F5
:10033000013983162206013C031DA429843083124F
:10034000BB060830BA068316A108031DAB29831229
:100350002E21C72983168312BD080319BC0ABD08C4
:100360000319B4290030B52901308316A200831285
:100370003C08053C0319BE290030BF290130831613
:100380002205003A0319C829831235212E2183162C
:10039000831235210310FE0C8316A00A75298312DF
:1003A0000034831686158312861D022B0130F4005B
:1003B000F430F3007408033C031CF429031DE42902
:1003C00073081F3C031CF4297408FD007308FC002B
:1003D00074088316A1007308A00083127120643092
:1003E000F3070318F40ADA290430FC00FA30FD00A0
:1003F0009D20FC0BF6298316061383120613831621
:10040000861383128613831606128312061283162E
:100410008612831286128316861283128612831620
:100420000612831206160430FC00FA30FD009D20EF
:10043000FC0B152A831606128312061283168612E7
:10044000831286120430FC00FA30FD009D20FC0B64
:10045000242A83160612831206128316861283122A
:1004600086160430FC00FA30FD009D20FC0B332A78
:1004700083160612831206128316861283128612C0
:100480000430FC00FA30FD009D20FC0B422A0330B2
:10049000FD007030FC008316A1016430A0008312BF
:1004A00071200430FC00FA30FD009D20FC0B532A23
:1004B0008316861383128613831606138312061778
:1004C0000430FC00FA30FD009D20FC0B622A8316EC
:1004D00006138312061383168613831286130430C1
:1004E000FC00FA30FD009D20FC0B712A83160613D8
:1004F0008312061383168613831286170430FC00BA
:10050000FA30FD009D20FC0B802A8316061383120F
:10051000061383168613831286130430FC00FA3008
:10052000FD009D20FC0B8F2A0330FD007030FC0085
:100530008316A1016430A000831271200430FC00F6
:10054000FA30FD009D20FC0BA02A8316861383122F
:1005500086138316061383120617831686128312D8
:10056000861283160612831206160430FC00FA3037
:10057000FD009D20FC0BB72A831606138312061379
:1005800083168613831286138316061283120612AD
:1005900083168612831286120430FC00FA30FD00A6
:1005A0009D20FC0BCE2A8316061383120613831696
:1005B0008613831286178316061283120612831679
:1005C0008612831286160430FC00FA30FD009D204E
:1005D000FC0BE52A83160613831206138316861373
:1005E000831286138316061283120612831686124E
:1005F000831286120430FC00FA30FD009D20FC0BB3
:10060000FC2AD129831606158312061DC22B8316D8
:1006100005168312051A1A2B0430FD004C30FC001D
:100620008316A1016430A000831271203230FD00D6
:100630009D20072B003083169C1B0130FC007C0D95
:10064000F700F70DF70DF830F70583121F08C739CB
:1006500077049F000630F700F70B2C2B00001F15C6
:100660001F19302B1E08F600003083161C1B0130AA
:10067000FC007C0DF700F70DF70DF830F70583123D
:100680001F08C73977049F000630F700F70B462B89
:1006900000001F151F194A2B1E08F5004830F000F6
:1006A0004C308316A0008312B2203A308316A0008B
:1006B0008312B22020308316A0008312B220750866
:1006C000FD001830FE00D3200530FC007C083720E8
:1006D000FC0AF7008316A0008312B2200A307C02C5
:1006E000031D662B7608FD001830FE00D32048302D
:1006F000FC003910FF30BB00BA00BC010130BD0066
:10070000BE01BF013F08093C031C8B2B7E30FE005D
:100710007321BF0A822BBD01BF013F080F3C031CA0
:100720009A2B29303F0784000008FD00FE0073214A
:10073000BF0A8D2BBF017C08840000080319A92B78
:100740007C0884000008FD00FE007321FC0ABF0A3B
:100750009B2B0130BE00FF30BA06BB063A08FE00F4
:1007600073213B08FE007321BE010130BD007E30C5
:10077000FE0073210430FC00FA30FD009D20FC0BCC
:10078000BC2B022B8A15BA28C10183169C1FCB2BC8
:100790008312C10A831600301C1B0130F7000310BE
:1007A000F70D77088312C104C108031DB12CF601AF
:1007B000F5014508023A0319E42B033A0319F72B14
:1007C000023A03190A2C212C8316861383128613EE
:1007D0008316061383120617831606128312061257
:1007E00083168612831286160130C500212C8316CB
:1007F0008612831286128316061283120616831639
:10080000061383120613831686138312861702308B
:10081000C500212C831686128312861283160612B7
:100820008312061683160613831206138316861385
:10083000831286170230C5003A30F6009830F50072
:10084000212C003083169C1B0130FC0000301C1B47
:1008500001307C04003A031D6D2C7508303C031DEB
:10086000672C7608753C031D672CF601F501831291
:100870004508023A0319402C033A0319532C662CFD
:1008800083168613831286138316061383120617A4
:100890008316061283120612831686128312861698
:1008A0000130C500662C83168612831286128316C9
:1008B0000612831206168316061383120613831676
:1008C0008613831286170230C500662C8316F50A3C
:1008D0000319F60A8312212C831683124508023A63
:1008E0000319762C033A0319892C9C2C8316861342
:1008F00083128613831606138312061783160612B5
:100900008312061283168612831286160130C500E2
:100910009C2C83168612831286128316061283126B
:100920000616831606138312061383168613831284
:1009300086170230C5009C2C3230FD009D208316A6
:1009400006138312061383168613831286138316E7
:100950000612831206128316861283128612033041
:10096000C100003483160613831206138316861300
:1009700083128617831606128312061283168612B6
:1009800083128616C830FD009D208316061283123E
:10099000061283168612831286128316061383129A
:1009A000061383168613831286130330FD008430EA
:1009B000FC0003308316A100E830A00083127120F0
:1009C0000330C500C4238316061283120612831651
:1009D0008612831286168316861383128613831655
:1009E000061383120617D730FD009D20831686124A
:1009F0008312861283160612831206168316861336
:100A00008312861383160613831206170330F5002C
:100A1000C830FD009D20F50B082D831606138312A8
:100A2000061383168613831286173230FD009D202D
:100A300083160613831206138316861383128613F6
:100A400083168612831286128316061283120616E6
:100A50000530F5006E30FD009D20F50B2A2D831624
:100A600086128312861283160612831206168316C6
:100A700086138312861383160613831206176430B7
:100A8000FD009D200230F4005830F300F308031DF0
:100A90004C2DF40803196B2DC10183169C1F532D97
:100AA0008312C10A831600301C1B0130F7000310AB
:100AB000F70D77088312C104C1080319632D323082
:100AC000FD009D206B2D0130FD009D207308031952
:100AD000F403F303462D83160612831206128316BF
:100AE0008612831286160230F4005830F300F308A1
:100AF000031D7D2DF4080319982DC10183169C1F39
:100B0000842D8312C10A831600301C1B0130F700AC
:100B10000310F70D77088312C104C108031D982D37
:100B20000130FD009D2073080319F403F303772DB2
:100B300083160612831206128316861283128612F9
:100B400083160613831206138316861383128613E5
:100B50000130C500C4235530C700C6018A15F728E7
:100B600083160613831206138316861383128613C5
:100B700083160612831206128316861283128612B9
:100B80000330FD002030FC0001308316A100F4305A
:100B9000A000831271204508023A0319D62D033AAA
:100BA00003190E2E023A0319462E482E0230F40085
:100BB0008A30F300F308031DE02DF4080319FD2D1E
:100BC00001084202031CED2D831606128312061241
:100BD0008316861283128616F52D8316061283124B
:100BE000061283168612831286120130FD009D20A4
:100BF00073080319F403F303DA2D83160613831223
:100C00000613831686138312861383160612831225
:100C100006128316861283128612482E0230F400C2
:100C20008A30F300F308031D182EF4080319352E3B
:100C300001084202031C252E831606138312061395
:100C400083168613831286172D2E8316061383129E
:100C5000061383168613831286130130FD009D2030
:100C600073080319F403F303122E83160613831279
:100C700006138316861383128613831606128312B5
:100C800006128316861283128612482E6A2E482E6A
:100C90000330FD002030FC0001308316A100F43049
:100CA000A000831271208316861283128612831687
:100CB0000612831206168316861383128613831672
:100CC0000613831206170230F500AF30FD009D2099
:100CD000F50B652E831606138312061383168613EF
:100CE0008312861383160612831206128316861247
:100CF000831286120330C500C4235530C700C601D5
:040D00008A15902997
:1010000084011F30830583161F129F121B0880392D
:101010009B0007309C001C0883120D136030831660
:101020008F0082308312A9009830AA00AB004030B4
:10103000AC00AD00AE006030AF008630B000B43020
:10104000B1006030B200A430B300B400B50061302C
:10105000B6000330B700F030B800F0018316061375
:1010600083120613831686138312861383160612C1
:10107000831206128316861283128612623083163A
:101080008F008113831294128316061186140612A0
:10109000003083129400831694000108C739083881
:1010A00081004830F800053883129200FF30831623
:1010B00092001F129F121B08803904389B001F13D7
:1010C00083121F179F1783169F1383121F1410304C
:1010D000F8001F08C73978049F00853090008316F8
:1010E00086150B3083129700960107309500023069
:1010F00083169C000508033885000330F700F70BC2
:101100007F281C0883120D138A3083169D0003303C
:10111000FD00E830FC00A101C830A0008A11831254
:1011200071208A153230FD008A119D208A15033006
:10113000FD00E830FC008316A101C830A0008A1130
:10114000831271208A150430F300FA30FD008A11F1
:101150009D208A15F30BA52883168C14C0308312AA
:101160008B040330C000C100C400C500E630C200DB
:101170008A11D1298A158A11C4238A150230F300F5
:10118000FA30FD008A119D208A15F30BC028033028
:10119000FD00E830FC008316A101C830A0008A11D0
:1011A000831271208A150230F300FA30FD008A1193
:1011B0009D208A15F30BD528C00183169C1FE328B8
:1011C0008312C00A831600301C1B0130F700031085
:1011D000F70D77088312C0041F19EC281E087F3C06
:1011E000031CF828C708031DF8288A11B22C8A1599
:1011F0004008033A03190329013A03191729033A4E
:10120000031950298929831686138312861383169E
:10121000061383120617831686128312861283160C
:10122000061283120616C6010330C500DC28010829
:10123000F300E63043077302031920290318292914
:1012400083168613831286138316061383120617DA
:10125000312983160613831206138316861383120D
:1012600086130108F300F0304307730203193A298B
:1012700003184329831686128312861283160612D8
:10128000831206164B298316061283120612831642
:101290008612831286120230C100C601C500DC2806
:1012A0000108F300E63043077302031959290318B4
:1012B00062298316861283128612831606128312FF
:1012C00006166A29831606128312061283168612E0
:1012D000831286120108F300F030430773020319EA
:1012E000732903187C2983168613831286138316A9
:1012F0000613831206178429831606138312061316
:1013000083168613831286130130C100C601C500FF
:10131000DC28C3014608543C031891298A11B02DDA
:101320008A1541084402031999294108C400C830AC
:10133000C2004108023C031DBD2983160613831217
:101340000613831686138312861301084202031CB8
:10135000B22983168612831286128316061283120E
:101360000616BA29831606128312061283168612EF
:10137000831286120230C500DC29831606128312FE
:101380000612831686128312861201084202031C7B
:10139000D2298316861383128613831606138312AB
:1013A0000617DA298316061383120613831686138B
:0C13B000831286130130C500DC286300A6
:04400E00383FFC3FFC
:00000001FF
